:100000000C94E9000C9406010C9406010C94060172
:100010000C9406010C9406010C9406010C94060144
:100020000C9406010C9406010C9472180C9444195B
:100030000C9497130C9406010C9406010C94060181
:100040000C9406010C9406010C9406010C94060114
:100050000C9406010C941F140C9406010C940601D8
:100060000C9406010C9406010C9406010C940601F4
:100070000C9406010C9406010C9406010C940601E4
:100080000C9406010C9406010C9406010C940601D4
:100090000C9406010C9406010C9406010C940601C4
:1000A0000C9406010C9406010C9406011E031E0319
:1000B0004A034A03B203DD04DD04DD04D00369040E
:1000C0007A047A04B119D819D01AD819D01A241A76
:1000D000471AD01A9E1AAD1A3A003B003C00BC00E9
:1000E000AE00BB00A800AA00A900100347006500ED
:1000F00065006B00500061006400000010034200C6
:10010000540048004C0061006200730000000403CA
:10011000090409023B00020100A0FA0904000001E1
:10012000030101000921110100012240000705819E
:100130000308000109040100010300000009211166
:100140000100012232000705820320000112010094
:100150000200000008EDFE57420100010200010507
:10016000010980A101850319012AB700150126B7ED
:1001700000950175108100C0050C0901A1018504DD
:1001800019012AA002150126A0029501751081000F
:10019000C005010906A101050719E029E715002599
:1001A00001950875018102950175088101050719FE
:1001B0000029FF150026FF00950675088100050837
:1001C00019012905950575019102950175039101A4
:1001D000C00011241FBECFEFDAE0DEBFCDBF11E0BB
:1001E000A0E0B1E0E6EBF6E302C005900D92AA377D
:1001F000B107D9F722E0AAE7B1E001C01D92AD3105
:10020000B207E1F70E9478100C94591B0C9400007F
:1002100081E0089581E008950C940A0108950C94FA
:100220000E011F93CF93DF9300D000D01F92CDB764
:10023000DEB749835A836B8330917D0189819A812E
:10024000311114C0662359F0222349F00E94160789
:10025000182F682F89819A810E94BF0603C00E94CF
:10026000EA06182F69817A81812F04C00E9416073F
:1002700069817A810F900F900F900F900F90DF910E
:10028000CF911F910C941F0EFC01262F40815181AC
:100290006281738184810C94110181E00895CF9370
:1002A000DF93EC0160E00E944401BE01DF91CF9139
:1002B0000C940F010C944E0F0C944A0F08950E9459
:1002C00069050E945E012FEF84E39CE0215080408D
:1002D0009040E1F700C000000C9445140F931F9369
:1002E000CF93DF938C0161E00E944401EC01B801DF
:1002F0000E940C018823F1F1B801CE010E94711215
:100300008823C1F1B801CE010E948510882391F1A4
:10031000B801CE010E94CD11882361F1F8018281DC
:10032000882309F1CB358DE5D807C1F050F4C1150C
:10033000FCE5DF0781F0CF3DDC45A9F40E94470CC6
:1003400019C0CC35EDE5DE0761F0CD35DD4559F45A
:100350000E94900B08C00E945F010CC00E94990B84
:1003600002C00E949C0BC801DF91CF911F910F9199
:100370000C94080180E0DF91CF911F910F910895B7
:100380000E947A130C94D9010E94DC010C94801312
:1003900008950C94C80181E008950C94CB01089550
:1003A000CF93C82F0E94C9018C2F0E94CD01CF91FD
:1003B000089580E00C94D0010E94CD120C94D001DD
:1003C0000E94CD1290917C01891721F080937C01CD
:1003D0000C94D0010895CF93DF93CDB7DEB72B9760
:1003E0000FB6F894DEBF0FBECDBF4F835887698725
:1003F0007A878B8761110E94DC0A9E012F5F3F4F35
:1004000086E0F90111928A95E9F785E0FE013796B9
:10041000D90101900D928A95E1F789819A814C81E9
:100420005D81452B31F09F3F31F491E08F3F19F40E
:1004300003C091E001C090E090FF09C049815A815A
:100440006B817C818D819E810E94FD0905C0C9015F
:100450000E944D018111F2CF2B960FB6F894DEBFAA
:100460000FBECDBFDF91CF910895FC0180819181B6
:100470000E9458070895CF93882309F448C0C82FD5
:100480008CEF8C0F813AD0F46C2F80910201909107
:1004900003010E941C13882349F06C2F80910201F4
:1004A000909103010E9454130E94FE0A6C2F8091C8
:1004B0000201909103010E9452130CC080E28C0F44
:1004C000883058F4C77081E001C0880FCA95EAF7F8
:1004D0000E94BF0ACF910C94FE0AEBE5EC0FE330CB
:1004E00040F4F0E0E15CFE4F808190E0CF910C940D
:1004F000E412C85AC73158F4EC2FF0E0EE0FFF1F9A
:10050000EF5EFE4F80819181CF910C94FA12CF91D2
:100510000895882349F1682F8CEF860F813A38F4CB
:1005200080910201909103010E9454130CC080E25B
:10053000860F883050F4677081E001C0880F6A959B
:10054000EAF70E94C50A0C94FE0A8BE5860F8330F9
:1005500020F480E090E00C94E412685A673120F4B3
:1005600080E090E00C94FA1208951F93CF93DF93EC
:10057000182FEB010E943B02209741F08FE99FE08A
:100580000197F1F700C000002197F6CF812FDF918E
:10059000CF911F910C948902893319F060E070E0CB
:1005A00002C060E570E00C94B502882321F00E943F
:1005B000BF0A0C94FE0A0895882321F00E94C50A00
:1005C0000C94FE0A0895CF92DF92EF92FF920F9360
:1005D0001F93CF93DF937C01D62FC72FFC0112818D
:1005E000058102950F700E94B50A8823B9F0112386
:1005F000A9F08C2F807F803421F080E28D0F88302D
:1006000068F08091050282FD09C082E00E945E0BC5
:100610000E94B50A91E0D82ED92601C0D12CCC2E4B
:10062000C2948FE0C8228C2D90E08C30910508F0A8
:10063000C4C1FC01EA5AFF4F0C94041B8C2F807F2D
:10064000CF70882311F0C295C07F112399F0CC237D
:1006500009F49FC180E28D0F883010F0D11104C0E1
:100660008C2F0E94BF0A03C08C2F0E94CF0A0E94C9
:10067000FE0A8FC18D2F0E948902CC2309F49DC1EF
:1006800080E28D0F883038F1DD2329F18C2F0E9414
:10069000D50A24C08C2F807FCF70803211F0C29594
:1006A000C07FDD2319F0D130A1F13DC0809105025A
:1006B00082FF17C0112349F0CC2329F08C2F0E9410
:1006C000BF0A0E94FE0A80E065C180E00E948902A4
:1006D000CC2309F472C18C2F0E94C50A0E94FE0A25
:1006E0006CC1112371F0002341F0013031F40E94FC
:1006F000DF0A8C2B0E94E70A60C10E94DF0A8C2B64
:100700001DC0002319F0013009F457C10E94F40AFA
:1007100025C0112321F0063008F04FC10EC005306E
:1007200008F04BC11BC0112361F0002331F0F70129
:10073000858180FF2EC18F7085838C2F0E94D5020A
:100740003CC1002359F0D93309F034C1FFEF07EE63
:1007500013E0F15000401040E1F72AC18C2F0E94B5
:10076000DC022BC18C2F86958695837019F0813021
:1007700061F023C1112321F08D2F9C2F937002C0B3
:1007800080E090E00E94E41220C1112321F08D2F1F
:100790009C2F937002C080E090E00E94FA1215C175
:1007A0008C2F837009F047C011110BC12D2F22959A
:1007B00026952770220F220F6D2F6F70862F90E0E5
:1007C000A0E0B0E0022E04C0880F991FAA1FBB1F33
:1007D0000A94D2F7D4FF10C04FE050E060E070E020
:1007E00004C0440F551F661F771F2A95D2F7409506
:1007F00050956095709503C040E050E0BA01C695F1
:10080000C695C3708A019B01082B192B2A2B3B2B01
:10081000C901B801C23049F058F4C13019F00E9442
:10082000D505CFC00E94C305CCC00E94E705C9C052
:100830000E94C105C6C0112319F08C2F817001C020
:100840008695882309F4BDC02D2F22952695277003
:10085000220F220F6D2F6F70862F90E0A0E0B0E086
:10086000022E04C0880F991FAA1FBB1F0A94D2F73B
:10087000D4FF10C04FE050E060E070E004C0440FCF
:10088000551F661F771F2A95D2F7409550956095A2
:10089000709503C040E050E0BA01C695C695C3709C
:1008A0008A019B01082B192B2A2B3B2BC901B8016C
:1008B000C23049F058F4C13019F00E949A0681C044
:1008C0000E9488067EC00E94AC067BC00E94FB0589
:1008D00078C0CF70112339F08C2F0E9421068D2F04
:1008E0000E94D5026EC08D2F0E94DC028C2F0E94C8
:1008F000420667C0D23F21F128F4D03F41F0D13FFA
:10090000C1F043C0D33F19F1D43F79F03EC0112369
:1009100041F0053008F051C08C2F8F710E9467069E
:100920004CC0063008F049C0F7CF8091050282FF25
:1009300018C0112339F08C2F8F710E9421063DC001
:100940001123C9F38C2F8F710E94420636C01123E8
:1009500029F08C2F8F710E940C062FC00E94070671
:100960002CC0112349F0CF718C2F0E94210663E027
:100970008C2F0E94430B21C081E00E945E0B02304D
:10098000E0F082E00E945E0B18C0112331F00023DA
:1009900091F28D2F0E943B0210C0002399F2D933AF
:1009A00049F41FEF27EE33E0115020403040E1F7CB
:1009B00000C000008D2F0E94890288EF8C0D8430CA
:1009C00020F40E94CD120E94D001DD20C9F00E94C7
:1009D000B10A80FD15C0F70112820E94AB0A0E9485
:1009E0002106C7010E9421050E94AB0ADF91CF9129
:1009F0001F910F91FF90EF90DF90CF900C944206E3
:100A0000DF91CF911F910F91FF90EF90DF90CF90EA
:100A100008950F931F93CF93DF93EC016881798141
:100A20008A810E9463078C010E94BE060E94AF0566
:100A3000B801CE010E94E302DF91CF911F910F9187
:100A40000895CF93DF93EC01988189812B813C81BC
:100A5000232B31F08F3F31F481E09F3F19F403C025
:100A600081E001C080E080FD1DC0CE010E946E01CA
:100A7000811110C00E94B50A8823A1F08A818823C1
:100A800089F08091050282FD0DC082E0DF91CF9157
:100A90000C945E0BCE010E940905CE01DF91CF912F
:100AA0000C944F01DF91CF91089580E090E00E9477
:100AB000E41280E090E00E94FA120E94DC0A0C949A
:100AC000FE0A80910201909103010E9456130C943A
:100AD00055050E94CC0A0C94610592959F70963042
:100AE00079F010F4925001C09A50923068F4803F2F
:100AF00069F018F4883E40F409C0843F29F406C028
:100B0000883E20F0813F11F080E0089581E0089553
:100B1000FC01808191810E9458070E946D05089513
:100B2000CF93DF9300D000D01F92CDB7DEB70F90E8
:100B30000F900F900F900F90DF91CF910895CF936A
:100B4000DF9300D000D000D0CDB7DEB726960FB629
:100B5000F894DEBF0FBECDBFDF91CF910895089509
:100B600008950C94B0050C94B1050E94B3056093F0
:100B70008C0170938D0180938E0190938F010C9462
:100B800055050C94B5050F931F9300918C0110919E
:100B90008D0120918E0130918F01602B712B822B62
:100BA000932B1F910F910C94B5050F931F930091F8
:100BB0008C0110918D0120918E0130918F01602365
:100BC0007123822393231F910F910C94B5050F93EA
:100BD0001F9300918C0110918D0120918E01309115
:100BE0008F0160277127822793271F910F910C9403
:100BF000B5050C94B0050E94F905609388017093C7
:100C0000890180938A0190938B010C94550560E0D3
:100C100070E0CB010C94FB050F931F9341E050E073
:100C200060E070E08A019B0104C0000F111F221FC9
:100C3000331F8A95D2F7C901B8011F910F910C9407
:100C4000FB050F931F9341E050E060E070E004C0AB
:100C5000440F551F661F771F8A95D2F78091880130
:100C600090918901A0918A01B0918B018A019B0129
:100C7000082B192B2A2B3B2BC901B8011F910F916F
:100C80000C94FB050F931F9341E050E060E070E08F
:100C900004C0440F551F661F771F8A95D2F74095F1
:100CA0005095609570958091880190918901A091EF
:100CB0008A01B0918B018A019B01082319232A2301
:100CC0003B23C901B8011F910F910C94FB050F93B1
:100CD0001F9341E050E060E070E004C0440F551FF6
:100CE000661F771F8A95D2F78091880190918901BC
:100CF000A0918A01B0918B018A019B0108271927D5
:100D00002A273B27C901B8011F910F910C94FB05BD
:100D10000F931F93009188011091890120918A01FE
:100D200030918B01602B712B822B932B1F910F9194
:100D30000C94FB050F931F9300918801109189017A
:100D400020918A0130918B016023712382239323A8
:100D50001F910F910C94FB050F931F930091880135
:100D60001091890120918A0130918B0160277127B0
:100D7000822793271F910F910C94FB050895292F2B
:100D8000220F920F890FE82FE695E695E69587707A
:100D900051E001C0550F8A95EAF785E0E89FF00120
:100DA0001124E258FE4F20E030E070E04081CB019A
:100DB000022E02C0969587950A94E2F7817081957C
:100DC00084278523842781932F5F3F4F253031056A
:100DD00069F70895292F220F920F890F682F6695C2
:100DE00066956695982F977085E0689FB0011124ED
:100DF00040E050E080E0FB01E40FF51FE258FE4FB9
:100E0000208130E0092E02C0369527950A94E2F73A
:100E100021703327042E01C0220F0A94EAF7822B97
:100E20004F5F5F4F4530510531F70895BF92CF9224
:100E3000DF92EF92FF920F931F93CF93DF938C017A
:100E4000C0908801D0908901E0908A01F0908B01D8
:100E500080918C0190918D01A0918E01B0918F01B4
:100E6000C82AD92AEA2AFB2ACFE1D0E0D701C60155
:100E70000C2E04C0B695A795979587950A94D2F73E
:100E800080FD04C0219790F7B12C07C0BC2EB8019B
:100E90008C2F0E94350E0197A9F38B2DDF91CF91F6
:100EA0001F910F91FF90EF90DF90CF90BF9008952A
:100EB000CF93DF93EC010E941607BE010E94350E0E
:100EC000DF91CF9108951F93CF93DF93EB01909122
:100ED0007D01992321F0CB010E94580713C088237C
:100EE00049F0CB010E941607182F682FCE010E94EF
:100EF000BF0604C0CB010E94EA06182FBE01812F55
:100F00000E94350EDF91CF911F9108951F93CF93CB
:100F1000DF93C091900116E080919101C81799F07C
:100F2000D0E01C9FF0011D9FF00D1124EE56FE4FE6
:100F30004081518162817381848195810E949F05E6
:100F40002196C770E9CFDF91CF911F91089540910D
:100F5000C2015091C3016091C4017091C50180919B
:100F6000C6019091C7010C949F05EF92FF920F93D9
:100F70001F93CF93DF938091C70182958F7009F003
:100F800065C08091C401882309F460C080919001FC
:100F9000F09091011091C2010091C3016091C501CF
:100FA0007091C60191E01F3F09F090E0C0910001EF
:100FB000D0910101292F96E0E92E8F1509F446C042
:100FC0006115710521F00F3F21F030E003C031E0E1
:100FD00001C0322F90E030FD36C0E89EF001E99E5E
:100FE000F00D1124DF01AE56BE4F11963C911197C2
:100FF000301329C03C91311326C012963C911297B0
:10100000311121C013964D915C911497461B570BDB
:101010004C175D07C0F48091C7018F708061809389
:10102000C701E956FE4F80818F708061808382EC1A
:1010300091E00E942105DF91CF911F910F91FF90C8
:10104000EF900C94860701968770B7CFDF91CF9110
:101050001F910F91FF90EF9008959F92AF92BF92D2
:10106000CF92DF92EF92FF920F931F93CF93DF9374
:10107000CDB7DEB761970FB6F894DEBF0FBECDBF18
:101080008C0185E0F801DE011D9601900D928A9594
:10109000E1F7D8011296EC909091C201E091C30162
:1010A0002091C5013091C6012115310531F0EF3F86
:1010B00031F481E09F3F19F403C081E001C080E07A
:1010C000B82FB1709B2E80FD47C1D8014C9111966D
:1010D0005C9111971396AD90BC90149782ECC82E3A
:1010E00081E0D82EF090C401B501621B730B2091F2
:1010F000000130910101FF2009F4D9C08091C7019E
:101100006217730708F095C0282F207F09F052C09E
:101110005E1313C0491311C0FE2CE1100EC08F7076
:1011200080618093C7010E94A707C6010E94210524
:101130008091C701F80185834DC1AB2831F05F3F35
:1011400031F481E04F3F19F403C081E001C080E039
:1011500080FD03C081E08E2502C080E090E0F82F82
:10116000F170FF2E80FF1CC08091900120919101B1
:1011700036E0821709F40BC190E0389FF001399FE7
:10118000F00D1124EE56FE4F6181561306C06081AA
:10119000461303C06281E61203C001968770E9CF4F
:1011A000FE2CEE2009F416C18091C7018160809366
:1011B000C70154C05E1306C0491304C0E11002C049
:1011C000F80199C0C8010E948805882361F1EE20CA
:1011D00051F12091C701822F82958F7090E0029784
:1011E00074F08091C2019091C30198878F83198612
:1011F000BB86AA862C87CE0107960E94210586E031
:10120000F801A2ECB1E001900D928A95E1F70E94FD
:10121000B5070E94A7070AC05E1711F1C8010E9416
:10122000880581112CC0C8010E942105FF24F39478
:10123000D1C0282F207F81F77A2DB98AA88A6E2DF8
:1012400089890E94900582EC91E00E94210586E048
:10125000D6011D928A95E9F70E94A707F12CBAC022
:101260004913DCCFE110DACFF8018583C8010E9471
:10127000210586E0D6011D928A95E9F7ABC0EE20E4
:1012800091F22091C701822F82958F7090E0029792
:101290000CF4B5CF8091C2019091C3019A838983E8
:1012A0001B82BD82AC822E83CE010196A6CF62172F
:1012B000730708F044C0FE2CEE2009F4B4CF5E138F
:1012C00030C049132EC02091C70120FD21C0822FBC
:1012D00082958F70482F50E041155105C9F0F801F3
:1012E00025834F30510541F08F5F982F9295907F65
:1012F000822F8F70892B8583C8010E94210586E08B
:10130000F801A2ECB1E001900D928A95E1F73CC0A2
:1013100086E0F801A2ECB1E001900D928A95E1F728
:1013200059C0C8010E948805811169CF8091C70109
:1013300081608093C701C8010E9421054BC07A2DAE
:10134000B98AA88A6E2D89890E94900586E0D60107
:101350001D928A95E9F718C0EE2009F464CFC80100
:101360000E948805F82E882309F45DCF86E0F801F5
:10137000A2ECB1E001900D928A95E1F782EC91E048
:101380000E9435020E94B5070E94A70723C04D871F
:101390005E878D859E850E945807292F22952F7084
:1013A000223028F49F7039F0811105C00BC0243021
:1013B00028F49F7049F4805E883020F0C8010E94B4
:1013C00021059F2CF92C06C0D80115969C91907F81
:1013D00091F7F8CF8F2D61960FB6F894DEBF0FBE50
:1013E000CDBFDF91CF911F910F91FF90EF90DF90D4
:1013F000CF90BF90AF909F9008951F93CF93DF93AE
:10140000CDB7DEB72C970FB6F894DEBF0FBECDBFB9
:101410004F83588769877A878B879C87CE01079689
:101420000E942D088823D1F09F8188852A853B85DD
:10143000232B31F08F3F31F481E09F3F19F403C03B
:1014400081E001C080E080FD47C04F8158856985FB
:101450007A858B859C850E949F053EC086E0FE01B3
:101460003796DE01119601900D928A95E1F7FF8182
:10147000E8856A857B856115710531F0EF3F31F4B0
:1014800081E0FF3F19F403C081E001C080E080FDEE
:1014900023C02091910130E0C901019687709927FE
:1014A0004091900150E084179507F1F1F983EA83A8
:1014B0007D836C8396E0929FD001939FB00D1124A1
:1014C000AE56BE4FFE01319601900D929A95E1F70E
:1014D000809391010E94860716E08091900190917F
:1014E0009101891771F1189FC00111248E569E4FEA
:1014F0000E942D08882329F1E09190011E9FF001A0
:101500001124EE56FE4F40815181628173818481A6
:1015100095810E949F058091900190E001968770CF
:10152000992780939001D9CF0E946905109291016B
:1015300010929001E2ECF1E086E0DF011D928A95C5
:10154000E9F72C960FB6F894DEBF0FBECDBFDF9142
:10155000CF911F9108958091D001859585958595AE
:1015600008958091D001877008959091D00197706F
:1015700081E009F480E008958091DB010895909165
:10158000DB01892B8093DB01089580959091DB012D
:1015900089238093DB0108951092DB0108959091D7
:1015A000DA01892B8093DA01089580959091DA0110
:1015B00089238093DA0108951092DA0108958091C9
:1015C000D101089508950C94E20A0C94E30A9091D5
:1015D000050292FD08C09091D101981721F08093E7
:1015E000D1010C94E50A08958091D101882329F056
:1015F0001092D10180E00C94E50A0895CF93DF9317
:10160000E0910201F09103018091DB018083E09180
:101610000201F091030190818091DA01892B80838E
:101620008091D101882381F0E0910201F0910301C2
:101630009081892B808380910201909103010E9407
:10164000101381110E94F40AC0910201D09103018C
:1016500048E050E068EC71E0CE010E940A1B892B43
:1016600069F088E0FE01A8ECB1E001900D928A9546
:10167000E1F7CE01DF91CF910C94D912DF91CF9198
:1016800008950C94E20A9091050292FD10C098E032
:10169000899F90011124262B2093D0010E942106BE
:1016A0008091D0018595859585950C94410B0C947E
:1016B00021061092D00180E00C94410B2091D001C2
:1016C000809582238093D001982F977099F430E011
:1016D000482F082E000C550B2417350759F0909110
:1016E000050292FD07C08595859585950E94420665
:1016F0000C94590B08959091050292FB222720F932
:10170000281769F080FB92F99093050280910402FA
:10171000909105020E94C30B82E00C945E0B089529
:101720008091050282FB882780F991E089270C943B
:101730007B0B81E00C947B0B80E00C947B0B80E0B6
:1017400090E00E941F1B21E0893E9E4F09F020E09F
:10175000822F089582E090E00C94171B83E090E0C4
:101760000C94171BCF9384E090E00E94171BC82FA6
:1017700082E290E00E94171B2C2F30E0A901582B29
:10178000CA01CF910895CF93C92F682F84E090E0CC
:101790000E94251B6C2F82E290E0CF910C94251BB8
:1017A000AB01BC018FE090E00C94371BAB01BC0196
:1017B00083E190E00C94371B60E070E0CB010C9467
:1017C000D60B60E070E0CB010E94D00B0C94DC0BD8
:1017D00069EE7EEF80E090E00E94431B60E082E0D3
:1017E00090E00E94251B60E083E090E00E94251BB2
:1017F00010928C0110928D0110928E0110928F0127
:1018000060E084E090E00E94251B60E082E290E0CE
:101810000E94251B60E085E090E00E94251B60E0AF
:1018200086E090E00E94251B6FEF87E090E00E9429
:10183000251B40E050E0BA0188E090E00E94371B91
:1018400060E08DE090E00E94251B40E050E0BA018E
:1018500088E190E00E94371B60E087E190E00E9401
:10186000251B40E050E0BA018CE190E00E94371B5C
:1018700060E070E080E290E00E94431B40E050E0B6
:10188000BA0188E190E00E94371B0C94E10B0C94A4
:10189000E80B682F8EE090E00C94251B0E94041446
:1018A0006093E3017093E4018093E5019093E60176
:1018B0006093DF017093E0018093E1019093E20176
:1018C000089585B7806885BF85B7806885BF08950E
:1018D00081E008950C94680C08950C946C0C0C94A1
:1018E0006C0C0C946F0C0C946C0C0C94730C0C948E
:1018F0006C0C0E94610C81E19FE00E94C3120E9467
:10190000770C0C94750C0E946D0C0C946C0C0E945E
:10191000140F0C94CF010E94EF130E94DD0F0E9460
:10192000870C0C94710C8F929F92AF92BF92CF92C2
:10193000DF92EF92FF920F931F93CF93DF93CDB778
:10194000DEB72A970FB6F894DEBF0FBECDBF0E9458
:10195000F20F982E81110E944E0C8CEDA82E81E082
:10196000B82E00E010E0802E802F0E94380FD82E75
:10197000F501C1905F01C826B1F40F5F1F4F03301E
:10198000110589F78FEF89838A831B820E94F813E0
:101990008160782F9D838C8349815A816B818D81F1
:1019A0000E94EB012FC08091E70181FD0E943E0F54
:1019B000E12CFF24F3948C2D8F21F1F00E946A0C0E
:1019C000882399F0EE828F82DF2081E009F480E0A5
:1019D00088870E94F8138160782F9A8789874E81C3
:1019E0005F8168858A850E94EB01F801E452FE4F11
:1019F0008081F826F08206C0E394FF0CF3E0EF123A
:101A0000DACFBBCF81E0911001C080E02A960FB6FB
:101A1000F894DEBF0FBECDBFDF91CF911F910F9124
:101A2000FF90EF90DF90CF90BF90AF909F908F90FE
:101A300008950E94930C0C94E001CF93DF930E94D1
:101A40003A0EEC01811522E59207E8F5811531E5A2
:101A5000930708F0B6C0883E910528F5803E9105B1
:101A600008F0E9C0883A910570F4853A910508F0CC
:101A70007AC08130910509F473C008F4D9C0049785
:101A800008F0D9C0D5C08F3B910508F0D1C0C85A25
:101A9000D0E0CC0FDD1FCE5BDE4F0990D881C02D8A
:101AA000CE019464C9C0811540E5940708F069C06F
:101AB000811550E4950708F060C09A9581159F4103
:101AC00008F4B9C0B5C0811536E5930728F581152E
:101AD00045E5940708F092C0811554E5950708F094
:101AE00087C0AC0143705527282F26952695C11530
:101AF000D34508F06CC081E090E002C0880F991FC8
:101B00004A95E2F740E2249F90011124EC01C22B98
:101B1000D32BCE019C6890C081152AE5920780F4F2
:101B2000811539E5930708F072C0811548E59407DF
:101B300008F47EC0D82FCC27CE01806F906A7CC07D
:101B400090568115904208F073C08D2F8F710E94BE
:101B5000CE0EDD27D0628F71AE01582BCA016CC04A
:101B600081E090E069C0C55AD0E0C059DE4F88815D
:101B7000C82FD0E0CE0190645FC0DF70CE01906AC4
:101B80005BC074E0969587957A95E1F7282F2370CE
:101B90003C2F337081E090E002C0880F991F3A9586
:101BA000E2F79C68AC01522B9A019C2F9F7096958E
:101BB000969550E2959FE0011124C9018C2B9D2B35
:101BC0003BC0D82FCC27CE01816F906A35C081E011
:101BD00090E002C0880F991F4A95E2F750E2259FD6
:101BE00090011124EC01C22BD32BCE019A6824C0A2
:101BF000D82FCC27CE01846F906A1EC00E94CE0ED3
:101C00008F7190E0D82FCC27CE01906215C08F70D5
:101C10000E94CE0E94E0D695C7959A95E1F7CF70C5
:101C2000D0E0DC2FCC27D0699E01282BC90104C04D
:101C300080E090E001C0CE01DF91CF910895272F81
:101C400030E0F901EE0FFF1F2E0F3F1FF90199E061
:101C5000899FE00DF11D1124E60FF11DEE0FFF1F0E
:101C6000E852FF4F8591949108950E941F0E0E94A3
:101C70001D0D08958238910569F1B0F48133910505
:101C800009F46DC048F48932910509F463C08A32C1
:101C9000910509F469C008958533910509F455C08B
:101CA00089339105B9F00895833E910569F138F4BF
:101CB000803E9105B1F0823E910509F10895863E7E
:101CC0009105A9F1873E9105B9F1843E910509F08E
:101CD00064C023C02091040220FD4FC021FD4DC0EF
:101CE00008958091040280FD44C08091050280FF28
:101CF00044C08091040284FD42C083EE4DC08091B7
:101D0000040282FF38C0F5CF8091040282FD33C007
:101D10008091050280FD31C0ECCF8091050281FFEA
:101D200032C08091040284FD2AC087EE35C08091C4
:101D3000040283FF26C0F5CF8091040283FD21C0F9
:101D40008091050281FD1FC0ECCF8091040285FDCA
:101D50001CC01DC08091040285FD19C016C0809171
:101D6000040286FD16C017C08091040286FD13C0D0
:101D700010C089E311C082EE0FC080EE0DC080E07C
:101D80000BC086EE09C084EE07C089E205C085E37A
:101D900003C08AE201C081E390E0089590910402BB
:101DA00092FF0DC0282F2871283019F4877F846096
:101DB00006C0282F2471243011F48B7F886093FF94
:101DC0000DC0282F2871283119F4877E846106C040
:101DD000282F2471243111F48B7E88612091050213
:101DE00020FF0DC0382F3871383019F4877F81609B
:101DF00006C0382F3171313011F48E7F886021FF99
:101E00000DC0282F2871283119F4877E816106C002
:101E1000282F2171213111F48E7E886194FD877EF7
:101E2000089580E0089508950E949F0B811102C0DB
:101E30000E94470C0E94AA0B8093E7010E94B20BFC
:101E400090930502809304020E94130F0E94AE0B30
:101E5000682F70E080E090E00E94C10560918801E9
:101E60007091890180918A0190918B010C94F90500
:101E7000E82FF0E0E75FFD4F80810895089580EA44
:101E80008A95F1F7089500C008950C943F0F0895C6
:101E90000C94470F0C94480F0C94470F0C944C0F64
:101EA000F894E82FE295EF70F0E031A1282F2F7021
:101EB00081E090E001C0880F2A95EAF7982F90956D
:101EC000932391A392A1892B82A37894089584EF00
:101ED0000E94500F85EF0E94500F86EF0E94500F16
:101EE00084E90E94500F80E90E94500F81E90C9410
:101EF000500FCF92DF92EF92FF920F931F93CF93E9
:101F0000DF938C01C62FD0E0CE018A589E4F7C0112
:101F1000FC0190819F3F09F447C0D62EF894E92F29
:101F2000E295EF70F0E081A19F7021E030E001C008
:101F3000220F9A95EAF7822B81A382A1209528236C
:101F400022A378940E94430FE3E7F1E046E751E0D3
:101F500031E0C12C21912F3F89F0A22FA295AF70C3
:101F6000B0E090968C9190E02F7002C09595879587
:101F70002A95E2F780FD02C0832F01C080E0C82AC5
:101F8000330F4E175F0731F7F70180818F3F11F054
:101F90000E94500F61E0C11001C060E08D2D0E94D1
:101FA000450FC00FD11FC882DF91CF911F910F91B4
:101FB000FF90EF90DF90CF9008950E94670F83E02D
:101FC000E9E0F2E0DF01982F1D929A95E9F7E6E04B
:101FD000F2E0DF011D928A95E9F783E00E94351057
:101FE0000C945A011F93CF93DF9300D01F92CDB76B
:101FF000DEB719821A821B8260E0CE0101960E9430
:10200000790F61E0CE0101960E94790F62E0CE0166
:1020100001960E94790F43E050E0BE016F5F7F4F51
:1020200086E092E00E940A1B11E0009709F410E09C
:10203000892B49F089819A81AB8180930602909324
:102040000702A0930802212F43E069E072E086E0D6
:1020500092E00E9436100E945C01812F0F900F9039
:102060000F90DF91CF911F9108950895FF920F93E4
:102070001F93CF93DF938C01F62ED72FC42F2223EB
:1020800049F081E08093EA010E94F8139093E901FE
:102090008093E8018091EA018823C1F08091E801F2
:1020A0009091E9010E941014059780F0EF2DFD2F0B
:1020B000D8014C2F50E0CD01801B910B8417950760
:1020C0001CF48D918193F7CF1092EA01DF91CF91AB
:1020D0001F910F91FF9008950E94CA150E948B0CCA
:1020E0000C94D6150E94DA150E94190D0C94F41563
:1020F0000E9496130E94B1150E94790C0E946C10E8
:102100000E9472100E94830CFBCFCF93DF93EC01EF
:10211000FB018281882309F43CC1C430FDE5DF075F
:1021200060F4CB3F9CE5D90788F49E0122503C45E2
:102130002431310508F02EC109C0C236EDE5DE07B5
:1021400029F0C63AFDE5DF0709F024C10E94B20B71
:102150009093050280930402C1318CE5D80709F4FD
:10216000C6C008F042C0C930ECE5DE0709F49BC0E8
:1021700000F5C5308CE5D80709F485C078F4C33084
:10218000ECE5DE0709F478C008F07AC0C230DC451F
:1021900009F0F5C0809104028160EFC0C7309CE572
:1021A000D90709F478C008F07AC0809104028061F0
:1021B000E4C0CD30FCE5DF0709F487C058F4CB302C
:1021C0009CE5D90709F479C008F07BC0809104022E
:1021D00088606FC0CF30FCE5DF0709F480C008F0ED
:1021E00082C080910402877FC8C0CE3F9CE5D9079A
:1021F00009F471C000F5C531FCE5DF0709F485C0BD
:1022000068F4C3319CE5D90709F475C008F095C09E
:102210000E946905809104028F77AFC0CC3FFCE536
:10222000DF07A9F108F054C0CB3FDC4509F0A7C097
:102230008091050240C0C230EDE5DE0709F489C097
:1022400058F4C1158DE5D80709F45AC008F069C0E3
:102250008091050282602FC0C236EDE5DE0709F4E9
:102260007CC0C63AFDE5DF0709F481C0C330DD4517
:1022700009F085C080E06EC08091040282607DC05C
:102280008091040216C080910402886076C080911B
:10229000050282604FC08091040280626EC080910E
:1022A000040280646AC00E9469058091040280680B
:1022B00064C0846062C081603DC0809104028E7FF2
:1022C0005CC0809104028D7F58C08091040216C0CA
:1022D0008091050218C0809105028D7F2BC08091EE
:1022E00004028F7E4AC0809104028F7D46C0809197
:1022F00004028F7B42C080910402877F8B7F3DC0A8
:10230000809105028D7F8E7F15C08091040282FB33
:10231000222720F991E0922790FB82F990FB83F924
:102320002CC080910502982F909591708E7F892BFB
:1023300090FB81F98093050222C00E94690580917B
:10234000040287FB222720F991E0922790FB87F96E
:1023500014C081E00E94490C12C08091040284FBE9
:10236000222720F991E0922790FB84F906C0809102
:102370000402982F909590FB80F98093040280913D
:102380000402909105020E94C30B0E94690580E03F
:1023900001C081E0DF91CF910895CF93DF93863123
:1023A0009C4541F5EB010E94BC0A982F8A8120913F
:1023B000020130910301882379F09A7A81E009F4CF
:1023C00080E08093EB01911102C069E201C065E3F6
:1023D000C9010E9452130AC08091EB01811102C011
:1023E00069E201C065E3C9010E9454130E94FE0A1C
:1023F00080E001C081E0DF91CF9108950F931F939A
:10240000CF93DF93C42FD22FFC0182818823C9F0A0
:102410004093EE010E94F8139093ED018093EC013C
:1024200080E28C0F883008F057C0C77081E001C08F
:10243000880FCA95EAF7DF91CF911F910F910C9405
:10244000D5028091EE01481330C08091EC0190914B
:10245000ED010E941014883C910538F510E21D0F23
:10246000CD17B9F080E28C0F883040F4C77081E05E
:1024700001C0880FCA95EAF70E94DC02183028F5DF
:1024800081E09D2F977001C0880F9A95EAF70E940E
:10249000D502802F0E94CC021830F0F4D77081E072
:1024A00001C0880FDA95EAF70AC080E28C0F883005
:1024B00098F4C77081E001C0880FCA95EAF7DF91F0
:1024C000CF911F910F910C94DC02802FDF91CF915F
:1024D0001F910F910C94CC02DF91CF911F910F911E
:1024E00008950F939C01CB01243F4CE5340731F153
:1024F00088F4293DFCE53F07D9F02A3D4CE5340737
:1025000079F1283D3C45A9F506E221EE41EE68ED62
:102510007CE52BC0263FFCE53F07E1F0A8F0273F14
:102520003C4539F507E225EE46EE67EF7CE51DC038
:1025300007E225EE45EE69ED7CE517C006E221EEE7
:1025400040EE64EF7CE511C007E225EE44EE65EF56
:102550007CE50BC006E221EE42EE66EF7CE505C0AD
:1025600008E221E045EE6AED7CE50E94FE1180E084
:1025700008C0FC018281882319F01092EE0101C08D
:1025800081E00F91089590937B0180937A010895E3
:102590009093F4018093F3010895E091F301F09199
:1025A000F401309721F00190F081E02D099480E052
:1025B0000895E091F301F091F401309721F0028049
:1025C000F381E02D099408952091F1013091F201F9
:1025D0002817390771F09093F2018093F101E0918F
:1025E000F301F091F401309721F00680F781E02D9E
:1025F000099408952091EF013091F00128173907CF
:1026000071F09093F0018093EF01E091F301F0916C
:10261000F401309721F00084F185E02D09940895AC
:10262000FC01329697E080E0915029F0219122231D
:10263000D9F38F5FF9CF0895662349F0FC013296F4
:1026400008962191621729F0E817F907D1F780E081
:10265000089581E008959C01FC0132969FEF80E08F
:102660004191461789F09F3F19F4411101C0982FFD
:102670008F5F8630A9F79F3F39F0F901E90FF11D0F
:1026800097FDFA956283089508959C012A5F3F4F54
:10269000FC014281461301C0128201968217930702
:1026A000B9F708950C942B130C944513029626E069
:1026B000FC0111922A95E9F7089508950C945D1391
:1026C00083E08093F5010C945E13811102C081E0D8
:1026D00001C082E08093F5010C945E130C946513A5
:1026E00081E08093F5010C945E130C9470130895AF
:1026F0000C9477130C9478130C9477130C94771331
:102700000C947713CF930E947E130E94F20F0E94C5
:102710007C13C0E08C2F0E94380F811104C0CF5F62
:10272000C330C1F701C081E0CF91089508951F9291
:102730000F920FB60F9211248F939F93AF93BF9375
:102740008091F601811113C080910C0290910D02CD
:10275000A0910E02B0910F024196A11DB11D809370
:102760000C0290930D02A0930E02B0930F02BF9142
:10277000AF919F918F910F900FBE0F901F90189562
:1027800080911402843031F10E94C0011092F60150
:1027900020E488E190E00FB6F894A895809360005B
:1027A0000FBE2093600083B7817F846083BF83B7AF
:1027B000816083BF7894889583B78E7F83BF0FB67F
:1027C000F894A895809160008861809360001092D1
:1027D00060000FBE08950E9469050C94C40182E058
:1027E00084BD93E095BD9AEF97BD80936E000895E8
:1027F0002FB7F89480910C0290910D02A0910E02D7
:10280000B0910F022FBF08952FB7F89460910C027A
:1028100070910D0280910E0290910F022FBF0895CA
:102820009C014FB7F89480910C0290910D02A091F9
:102830000E02B0910F024FBF821B930B0895789444
:102840001F920F920FB60F9211248F939F93AF9305
:10285000BF9380910C0290910D02A0910E02B09155
:102860000F020196A11DB11D80930C0290930D02E1
:10287000A0930E02B0930F02BF91AF919F918F91E1
:102880000F900FBE0F901F90189587E797E79093D2
:102890000108809300089AE088E10FB6F894A895A3
:1028A000809360000FBE90936000FFCF8091020282
:1028B00008950895CF93DF9321E02093E9002FEF4F
:1028C0003091E800215035FD06C035ED3A95F1F71D
:1028D00000002111F5CF2091E80025FF14C0EC0184
:1028E00040E050E068E070E00E9466168091E800E9
:1028F0008E778093E80088E0FE01AAEFB1E00190B6
:102900000D928A95E1F7DF91CF9108958093F701B9
:102910007093F9016093F80180911402843001F5FD
:1029200082E08093E9008FEF9091E800815095FD5F
:1029300006C095ED9A95F1F700008111F5CF8091D1
:10294000E80085FF0DC040E050E063E070E087EFF5
:1029500091E00E9466168091E8008E778093E800EF
:102960000895BC0184E00C948614BC0183E00C94AF
:102970008614089580911302811109C00E94F717EF
:102980000E9454188091E20084608093E2000895D0
:102990001092130208950C9475136091100281E057
:1029A000611101C080E00C9460139091140281E0E9
:1029B000943009F080E0609110020C94651342E0BD
:1029C00061EC81E00E94701742E261EC82E00E94BB
:1029D00070179091140281E0943009F080E06091CA
:1029E00010020C946E1380911602833009F461C0BA
:1029F00030F4813071F0823009F49AC008958A3041
:102A000009F486C08B3009F46CC0893009F0A8C085
:102A100020C080911502813A09F0A2C08091E8009F
:102A2000877F8093E8008091190290911A02892B88
:102A300021F468E08AEF91E003C060E080E090E07C
:102A400070E00E94B1168091E8008B778093E800D7
:102A5000089580911502813209F082C08091190297
:102A600090911A02029708F07BC08091E800877F5E
:102A70008093E8008091E80082FD05C080911402F7
:102A80008111F8CF6DC02091F3008091F20090E0A9
:102A9000922B029731F48091F100813011F0863051
:102AA00021F48091F100809302028091E8008B77FD
:102AB00053C080911502813A09F052C080911902E9
:102AC00090911A02892B09F04BC08091E800877F12
:102AD0008093E8008091E80080FFFCCF8091100196
:102AE00036C0809115028132D9F5809119029091FA
:102AF0001A02892BA9F58091E800877F8093E8006E
:102B00000E94A51780911702809310010C9469050B
:102B100080911502813221F58091E800877F8093B2
:102B2000E8000E94A517809118028093030208957F
:102B300080911502813AA1F48091E800877F80930B
:102B4000E8008091E80080FFFCCF80910302809331
:102B5000F1008091E8008E778093E8000C94A5172F
:102B6000089584B7877F84BF0FB6F894A8958091A5
:102B70006000886180936000109260000FBE90E05A
:102B800080E80FB6F89480936100909361000FBEC7
:102B90000C9470130E94F7170E945418E2EEF0E0B4
:102BA00080818460808378940C94E91A84E091E0B9
:102BB0000C94C812809114028530A9F480911402FB
:102BC000853079F40E94C013809112028823B1F3FA
:102BD0000E948213882391F30E9450160E94690577
:102BE000EDCF0C94EB13089508950C94F715292F4D
:102BF000332723303105C9F060F42130310581F0ED
:102C00002230310509F044C08BE390E022E131E04D
:102C100043C021323105E1F02232310549F138C09B
:102C200082E190E02DE431E037C0992781309105B1
:102C300049F028F0029761F5EAEEF0E005C0EEE019
:102C4000F1E002C0ECEFF0E0849190E09F0124C03D
:102C50006115710541F061307105D1F489E090E0B2
:102C60002DE331E019C089E090E024E231E014C0A6
:102C70006115710541F06130710551F482E390E016
:102C80002FE531E009C080E490E021E931E004C0A3
:102C900080E090E020E030E0FA0131832083089565
:102CA00080E189BD82E189BD09B400FEFDCF80913C
:102CB000D8008F7D8093D8008091E000826080935F
:102CC000E0008091E00081FDFCCF0895CF92DF927B
:102CD000EF92FF920F931F93CF93DF93EC018B0141
:102CE0007A010E94C417811133C0E114F10439F054
:102CF000F70180819181081B190BC80FD91FC12CC6
:102D0000D12C0115110519F18091E80085FD16C03F
:102D10008091E8008E778093E800E114F10449F097
:102D2000F70180819181C80ED91ED182C08285E0D1
:102D30000FC00E94C417882321F30AC08991809391
:102D4000F10001501109FFEFCF1ADF0ADACF80E05E
:102D5000DF91CF911F910F91FF90EF90DF90CF9077
:102D6000089520911B0230911C022617370748F066
:102D70006115710539F42091E8002E772093E80061
:102D800001C0B901FC0120E06115710579F1809164
:102D900014028823F1F18530F1F18091E80083FD80
:102DA0003CC08091E80082FD2EC08091E80080FF49
:102DB000EBCF2091F3008091F20090E0922B61150F
:102DC000710551F08830910538F421912093F1007C
:102DD000615071090196F3CF21E0089709F020E0D6
:102DE0008091E8008E778093E800CECF2111CFCF7D
:102DF0000AC080911402882361F0853061F08091CF
:102E0000E80083FD0AC08091E80082FFF2CF80E0F5
:102E1000089582E0089583E0089581E00895209167
:102E20001B0230911C022617370748F06115710507
:102E300039F42091E8002E772093E80001C0B90111
:102E4000FC0120E06115710591F180911402882345
:102E500009F440C0853009F43FC08091E80083FD4B
:102E60003DC08091E80082FD2FC08091E80080FF86
:102E7000E9CF2091F3008091F20090E0922B611550
:102E8000710559F08830910540F424912093F100A8
:102E90003196615071090196F2CF21E0089709F04F
:102EA00020E08091E8008E778093E800CBCF21115D
:102EB000CCCF0AC080911402882361F0853061F084
:102EC0008091E80083FD0AC08091E80082FFF2CF84
:102ED00080E0089582E0089583E0089581E00895F8
:102EE000982F973068F59093E900981739F0709112
:102EF000EC002091ED005091F00003C0242F762FBC
:102F000050E021FD02C09F5FECCF3091EB003E7F8F
:102F10003093EB003091ED003D7F3093ED00309128
:102F2000EB0031603093EB007093EC002093ED00E8
:102F30005093F0002091EE0027FDE5CF80E008954A
:102F40008F708093E90081E008958091150287FFDA
:102F500011C08091E80082FD05C0809114028111AA
:102F6000F8CF11C08091E8008B770BC080911402DC
:102F7000882349F08091E80080FFF8CF8091E80035
:102F80008E778093E80008952091E4003091E50069
:102F900095E64091EC00842F817040FF23C0809122
:102FA000E80080FD1DC080911402882399F08530CF
:102FB00099F08091EB0085FD11C04091E4005091A3
:102FC000E5002417350729F3915011F09A01E1CF5C
:102FD00084E0089582E0089583E0089581E00895F3
:102FE00080E008954091E80042FFDDCF08950E94FF
:102FF00065180E946D18E0EEF0E0808181608083AA
:10300000E8EDF0E080818F77808319BCA7EDB0E018
:103010008C918E7F8C9380818F7E8083109213029F
:1030200008950F931F93CF93DF930E9465180E941A
:103030006D18C8EDD0E088818F778883888180689B
:10304000888388818F7D888319BC10921402109226
:103050001002109212021092110200EE10E0F8011C
:1030600080818B7F808388818160888342E060E0FB
:1030700080E00E947017E1EEF0E080818E7F808317
:10308000E2EEF0E0808181608083808188608083CF
:10309000F80180818E7F8083888180618883DF91C1
:1030A000CF911F910F910895E8EDF0E080818F7E20
:1030B0008083E7EDF0E080818160808384E082BFDF
:1030C00081E0809313020C941118E8EDF0E0808108
:1030D0008E7F80831092E20008951092DA001092A1
:1030E000E10008951F920F920FB60F9211242F93B3
:1030F0003F934F935F936F937F938F939F93AF9380
:10310000BF93EF93FF938091E10082FF0BC080910A
:10311000E20082FF07C08091E1008B7F8093E10095
:103120000E94E81A8091DA0080FF1FC08091D800C9
:1031300080FF1BC08091DA008E7F8093DA0080913F
:10314000D90080FF0DC080E189BD82E189BD09B44D
:1031500000FEFDCF81E0809314020E94BA1405C0E6
:1031600019BC109214020E94C8148091E10080FFE3
:1031700019C08091E20080FF15C08091E2008E7F2F
:103180008093E2008091E20080618093E200809170
:10319000D80080628093D80019BC85E08093140227
:1031A0000E94CD148091E10084FF30C08091E20044
:1031B00084FF2CC080E189BD82E189BD09B400FE95
:1031C000FDCF8091D8008F7D8093D8008091E10061
:1031D0008F7E8093E1008091E2008F7E8093E200F9
:1031E0008091E20081608093E20080911002882348
:1031F00011F084E007C08091E30087FD02C081E008
:1032000001C083E0809314020E94D5148091E100F4
:1032100083FF29C08091E20083FF25C08091E100F7
:10322000877F8093E10082E0809314021092100265
:103230008091E1008E7F8093E1008091E2008E7F9B
:103240008093E2008091E20080618093E20042E09E
:1032500060E080E00E9470178091F00088608093A9
:10326000F0000E94CB14FF91EF91BF91AF919F911D
:103270008F917F916F915F914F913F912F910F901F
:103280000FBE0F901F9018951F920F920FB60F92BE
:1032900011242F933F934F935F936F937F938F935B
:1032A0009F93AF93BF93CF93DF93EF93FF93C0911F
:1032B000E900CF708091EC00D82FD17080FDD0E86C
:1032C0001092E9008091F000877F8093F00078945D
:1032D0000E9488191092E9008091F0008860809324
:1032E000F000CD2BCF70C093E900FF91EF91DF91FB
:1032F000CF91BF91AF919F918F917F916F915F918E
:103300004F913F912F910F900FBE0F901F901895E6
:103310001F93CF93DF93CDB7DEB7AA970FB6F8947C
:10332000DEBF0FBECDBFE5E1F2E08091F1008193F9
:1033300022E0ED31F207C9F70E94F3148091E80012
:1033400083FF2EC18091150290911602492F50E003
:103350004A30510508F024C1FA01EE59FF4F0C9490
:10336000041B803821F0823809F01AC108C080910E
:10337000110290911202992389F082600FC080910E
:1033800019028F70873008F00BC18093E90080919B
:10339000EB0085FB882780F91092E9009091E80006
:1033A000977F9093E8008093F1001092F100D1C0D4
:1033B000282F2D7F09F0F4C0882319F0823061F0A6
:1033C000EFC080911702813009F0EAC0933009F014
:1033D00080E0809312022EC08091170281112AC0D2
:1033E000809119028F702FEF280F263008F0D8C077
:1033F0008093E9002091EB0020FF1CC0933021F462
:103400008091EB00806214C09091EB0090619093EA
:10341000EB0021E030E0A90102C0440F551F8A955E
:10342000E2F74093EA001092EA008091EB00886096
:103430008093EB001092E9008091E800877F8093F1
:10344000E8000E94A517ACC08111AAC01091170214
:103450001F778091E3008078812B8093E300809137
:10346000E800877F8093E8000E94A5178091E8001C
:1034700080FFFCCF8091E30080688093E30011110E
:1034800002C082E001C083E08093140289C08058AA
:10349000823008F085C080911702909118028C3D0F
:1034A00053E0950779F583E08A838AE289834FB7F1
:1034B000F894DE01139620E03EE051E2E32FF0E0C5
:1034C00050935700E49120FF03C0E295EF703F5FF7
:1034D000EF708E2F90E0EA3010F0C79601C0C096D2
:1034E0008D939D932F5F243149F74FBF8091E80062
:1034F000877F8093E8006AE270E0CE0101960E9427
:10350000B11616C06091190270911A02AE014F5F98
:103510005F4F0E94F515BC01892B09F441C09091C1
:10352000E800977F9093E80089819A810E940F17A5
:103530008091E8008B778093E80032C0803881F575
:103540008091E800877F8093E8008091100280934B
:10355000F1008091E8008E7772CF811121C08091B7
:1035600017029091180299270297D4F48091E800ED
:10357000877F8093E80080911702809310020E9459
:10358000A51780911002811106C08091E30087FD8C
:1035900002C081E001C084E0809314020E94DF1425
:1035A0008091E80083FF0AC08091E800877F8093C4
:1035B000E8008091EB0080628093EB00AA960FB642
:1035C000F894DEBF0FBECDBFDF91CF911F9108955C
:1035D0000895CF93809114028823A1F0C091E9004F
:1035E000CF709091EC00892F817090FD80E8C82BFE
:1035F0001092E9008091E80083FD0E948819CF7045
:10360000C093E900CF910895EE0FFF1F0590F4914C
:10361000E02D0994FB01DC0104C08D91019080191B
:1036200021F441505040C8F7881B990B0895F9992F
:10363000FECF92BD81BDF89A992780B50895A8E183
:10364000B0E042E050E00C944B1B262FF999FECFDE
:1036500092BD81BDF89A019700B4021639F01FBAE5
:1036600020BD0FB6F894FA9AF99A0FBE0895039602
:10367000272F0E94261B0E94251B252F0E94261BF8
:10368000242F0C94261B0196272F0E94261B0C9496
:10369000251BDC01CB01FC01F999FECF06C0F2BD70
:1036A000E1BDF89A319600B40D9241505040B8F700
:0636B0000895F894FFCF1D
:1036B600C800D20156145A14B914B514B1145914C9
:1036C60001E200E900EA00B500B600B700CD0083CC
:1036D60001CC008A019201940121022302240225D1
:1036E60002260227022A02B300B4006F007000818E
:1036F6008283E200E900EA00B500B600B700CD001B
:103706008301CC008A019201940121022302240242
:103716002502260227022A02B300B4006F007000B9
:0A372600818283949091F4F5F6007F
:00000001FF
